:020000006B296A
:08000800A1000308A0000B1188
:1000100020088300A10E210E09002208A300230856
:10002000233C031C1B282308113C031C1928053002
:100030002428093024282430A3022308113C031C5F
:1000400023280A3024280630A400271D4D28230821
:100050008207732878287F2886288B289228992859
:100060009E28A528AC28B128B828BF28C428CB28AA
:10007000D228D728DE28E528EA28F128F828FD2804
:1000800004290B29102917291E2923292A29312956
:1000900036293D294429492950292308820757290F
:1000A0005729572957295729572957295729572950
:1000B0005C295C295C295C295C295C295C295C2918
:1000C0005C296129612961296129612961296129E5
:1000D00061296129662966296629662966296629B2
:1000E0006629662966292408C038A600A500C32908
:1000F0002408C038A6002408D038A500C329240845
:10010000D038A6002408C038A500C3292408D03858
:10011000A600A500C3292408D038A6002408E0388A
:10012000A500C3292408E038A6002408D038A5007B
:10013000C3292408E038A600A500C3292408E03814
:10014000A6002408F038A500C3292408F038A6002A
:100150002408E038A500C3292408F038A600A5002B
:10016000C3292408F038A6002408B038A500C32904
:100170002408B038A6002408F038A500C3292408B4
:10018000B038A600A500C3292408B038A60024086A
:100190007038A500C32924087038A6002408B03898
:1001A000A500C32924087038A600A500C329240887
:1001B0007038A60024083038A500C3292408303838
:1001C000A60024087038A500C32924083038A600EA
:1001D000A500C32924083038A60024087038A500DB
:1001E000C32924087038A60024083038A500C32984
:1001F00024087038A600A500C32924087038A6007A
:100200002408B038A500C3292408B038A600240863
:100210007038A500C3292408B038A600A500C3295A
:100220002408B038A6002408F038A500C329240803
:10023000F038A6002408B038A500C3292408F038F7
:10024000A600A500C3292408F038A6002408E03839
:10025000A500C3292408E038A6002408F038A5002A
:10026000C3292408E038A600A500C3292408E038E3
:10027000A6002408D038A500C3292408D038A60039
:100280002408E038A500C3292408D038A600A5001A
:10029000C3292408D038A6002408C038A500C329E3
:1002A0002408C038A6002408D038A500C329240893
:1002B0009038A600A500C32924086038A600A50030
:1002C000C32924086038A600A500C3292408903853
:1002D000A600A500C329CD210D286B292708A80653
:1002E000281CBC29271CBC29271E9629A71D862946
:1002F000A71C8029A203A21FBC294730A200BC2949
:10030000A20A2208473C031CA201BC29A71C8F2972
:100310000330A202A21FBC294530A200BC29033031
:10032000A2072208453C031CA201BC29A71DAA293B
:10033000A71CA1290930A202A21FBC294330A20098
:10034000BC290930A2072208433C0318BC29043009
:10035000A200BC29A71CB3291230A202A21FBC29EB
:100360003F30A200BC291230A20722083F3C0318EC
:10037000BC290930A200BC292708A8000D2825089F
:1003800086000000000026088600000005082806F8
:100390000319BF292806A7006E298230831603138C
:1003A000810083120313831603139F018C018312B0
:1003B000031390019201970107309F0086010030DE
:1003C0008316031386008312031385011F308316DF
:1003D000031385008312031300308A002030840049
:1003E0008001840A0408803C031DF0290030A2002B
:0C03F0000508A700A80000308B000800E2
:02047C0000007E
:0204FE000000FC
:02057E0000007B
:0205FE000000FB
:02067C0000007C
:0206FE000000FA
:02077E00000079
:0207FE000000F9
:02087C0000007A
:0208FE000000F8
:02097E00000077
:0209FE000000F7
:020A7C00000078
:020AFE000000F6
:020B7E00000075
:020BFE000000F5
:020C7C00000076
:020CFE000000F4
:020D7E00000073
:020DFE000000F3
:020E7C00000074
:020EFE000000F2
:020F7E00000071
:020FFE000000F1
:02400E00223F4F
:00000001FF
